:1000000054C00BC2ECC3F8C36BC06AC069C068C0FF
:1000100067C066C065C064C063C062C00FC404032B
:10002000090422037700770077002E007200650034
:10003000630075007200730069006F006E002E008F
:100040006A00700010035500530042002D0032007A
:10005000330032001201100102000008C016E10551
:10006000000101020001090243000201008032097F
:100070000400000102020100052400100104240212
:100080000205240600010524010301070583030876
:1000900000FF09040100020A000000070501020236
:1000A0000000070581020800000011241FBECFE5F3
:1000B000D1E0DEBFCDBF10E0A0E6B0E0E4E9FBE0B8
:1000C00002C005900D92AC36B107D9F711E0ACE64D
:1000D000B0E001C01D92A034B107E1F7D2D458C5F9
:1000E0008FCF85B7826085BF8BB780648BBF8BE471
:1000F00080937D008093A8008AE580937C008093A4
:10010000A70008951F93CF93DF93DC01162FEA0118
:10011000888184FF05C0898198E88927898302C086
:100120008AE58883AE014E5F5F4F212FFA018D91E2
:10013000819321501216DCF3CA01612F57D11C5F45
:100140001883DF91CF911F91089547EA50E0DADFDD
:1001500008954CE750E0D6DF08951F93CF93DF93C7
:1001600060918D00635067FDB3C080918A00CCE040
:10017000D0E0C81BD109CF56DF4F80918900803174
:1001800018F4CE0162D49EC08D3209F08BC0683065
:1001900009F098C083EC809371008AE58093600039
:1001A00010926D008881807621F0CE0120D4282F16
:1001B00066C09A8110927A008981882321F4109276
:1001C0007B0022E055C0853019F490938E004FC01B
:1001D0008630B9F58B81813041F484E590E09093CD
:1001E0008C0080938B0022E128C0823021F4CE0164
:1001F000E9D3282F22C08330F9F48A81882341F47F
:100200008EE190E090938C0080938B0024E015C0E9
:10021000813041F482E290E090938C0080938B00D7
:1002200022E20BC0823041F484E490E090938C0091
:1002300080938B0020E101C020E080E480936D007A
:100240001EC0883021F421E080E990E013C089309D
:1002500019F4909390000BC08A3011F421E008C08B
:100260008B3029F48BE480937D008093A80020E0FC
:100270008AE790E090938C0080938B0009C02F3F19
:1002800039F4888187FD2E8180E880936D0006C057
:100290008F81882319F48E81821708F0822F809332
:1002A000610010C080916D0087FF0CC0CE012AD480
:1002B0008F3F21F48EE18093600004C0882311F009
:1002C0001092610080918D00181614F410928D0028
:1002D0008091600084FF58C0809161008F3F09F4D5
:1002E00053C0182F893008F018E0811B80936100FB
:1002F0008091710098E8892780937100112391F112
:1003000080916D0087FF08C082E790E0612F8ED357
:10031000182F893098F526C020918B0030918C00E1
:1003200086FF0DC0A2E7B0E080E090E0F901E80FA1
:10033000F91FE491ED9301961817C1F708C0912FAA
:10034000D901E2E7F0E08D9181939150E1F71150EE
:10035000812F90E01F5F0196820F931F90938C0076
:1003600080938B0082E790E0612F40D0612F6C5F1B
:100370006C3041F08FEF8093610004C08FEF809369
:1003800061006EE16093600094E186B3857031F4A2
:100390009150D9F710928E001092880010E09923A6
:1003A00009F411E080916C00811739F0112319F4E0
:1003B000F894A8D1789410936C00DF91CF911F919D
:1003C0000895A82FB92F80E090E041E050EA6095B1
:1003D00030E009C02D9182279795879510F08427EA
:1003E0009527305EC8F36F5FA8F30895EADF8D9319
:1003F0009D930895A6E088279927AA9569F001970B
:10040000E1F3B099FCCFB09BFECF81E09927A6B372
:10041000019611F0A570D9F70895CF93CFB7CF9378
:10042000C395B09BE9F7B09B0BC0B09B09C0B09BD4
:1004300007C0B09B05C0B09B03C0B09B01C0D8C033
:100440000F92DF93C0918A00DD27CF56DF4F012E38
:10045000B09B03C0DF910F90E6CF2F930F931F93B4
:100460004F932FEF4F6F06B300FB20F95F933F933D
:1004700050E03BE065C016B30126502950FDC895F9
:1004800056B3012700FB25F92F7306B3B1F05027AF
:10049000102710FB26F906B22230F0F000C016B388
:1004A000012700FB27F90126502906B22430E8F580
:1004B0004F77206816B30000F6CF50274F7D20629B
:1004C00006B2102F000000C006B3002650291027E6
:1004D00010FB26F906B2E2CF4F7B06B3206400C0C2
:1004E000DACF01265029157006B269F14E7F2160DE
:1004F000012F16B328C0002650294D7F06B2226076
:10050000102F29C0012650294B7F06B22460012FED
:100510002DC016B301265029477F2860000006B27F
:100520002EC04F7E06B3206130C0422706B34993E8
:1005300000265029102706B24FEF10FB20F9297F23
:1005400016B379F2157059F10126502906B2012728
:1005500000FB21F9237F06B371F2002650293150A8
:10056000D0F006B2102710FB22F9277E16B351F205
:1005700001265029012700FB06B223F92F7C49F2FE
:10058000000006B3102710FB24F90026502906B2FC
:100590002F7939F270CF10E41ABF00271CC03B50EE
:1005A0003195C31BD04010E41ABF0881033C21F1F0
:1005B0000B3411F1209188001981110F1213EDCF26
:1005C0004A81441F093669F10D3211F0013E29F7C5
:1005D0004F7009F0042F00938F003F915F914F916E
:1005E0001F910F912F91DF910F90CAB7C6FD18CFC1
:1005F000CF91CFBFCF91189520918F00222369F31F
:1006000010918D001123D1F53430D2F130938D004B
:100610002093890010918A003BE0311B30938A00BF
:100620002FC000918D0001304CF50AE54F7049F460
:100630003091600034FD25C000936000C1E7D0E038
:1006400024C0433049F030917C0034FD1AC000933F
:100650007C00CDE7D0E019C03091A70034FD11C077
:100660000093A700C8EAD0E010C0052710E000C042
:1006700021C0052710E0C89508BB14C03AE501C0A9
:1006800032ED032EC0E0D0E032E017B31560C09A1F
:1006900008B317BB55E020E84FEF20FF052708BB44
:1006A000279517951C3F28F700004552B0F720FF0B
:1006B0000527279508BB17951C3FB8F629913A9551
:1006C00061F70A7F10918E00110F08BBC250D04015
:1006D00011F01093880010E41ABF016017B31A7F5D
:1006E000402F4A7F54E05A95F1F708BB17BB48BB2F
:1006F00074CF80E090E036D28F3F11F481B78C5FE9
:1007000081BF0895CF92DF92EF92FF920F931F93D4
:10071000CF93DF93E1B66EDE6C0188E981BF6ADEBC
:100720008453994014F400E801C000E080E4F82EFE
:10073000C0E0D0E0102F1F0D11BF5CDE9C0189E0EE
:10074000243338070CF0102FF6942196C730D105CA
:1007500011F0012FEFCF2453394037FF03C03095FC
:1007600021953F4FC6018453994097FF03C0909550
:1007700081959F4F8217930714F4E1BE27C0125052
:1007800011BF1E5F7901C12FD0E0229610C032DE6A
:100790008453994097FF03C0909581959F4F8E1584
:1007A0009F0514F411B77C0181B78F5F81BF81B7BA
:1007B00090E0C817D9075CF711BF80E090E0D2D174
:1007C000811721F080E090E0612FD4D1DF91CF91AB
:1007D0001F910F91FF90EF90DF90CF900895B59902
:1007E000189501BB05B50FBD09E00DBD07E000BFC1
:1007F00000E40BBF01B3189501BB0FB702BB0DB5E9
:100800000A950DBD79F00BB50695B59900680BBD3D
:1008100013BB0FB51EB5011B0FBD13B302B30FBF42
:1008200001B3189500BF04BD0BB50DBB00E20ABFB4
:1008300000E60BBF02B30FBF01B3189501BBF099DF
:1008400007C00BE40EB90EBB08B50FB901B318957C
:1008500000E40EB900E003BF01B31895881F979517
:10086000881F9795881F9795881F9795881F97953C
:10087000881F9795881F9795881F9795892F0895AA
:100880009C0181E080BD80E888B9B99ABD988BB79A
:100890008F7D8BBF1ABC13BE10BE80EE8EB984E56F
:1008A0008DB98FEF8FB9B9017695679580E090E0AB
:1008B0006C5E70418C4F9F4F40E050E031D1215031
:1008C0002EBD8EB589BD1DBC8EB590E00196959567
:1008D000879595958795819585BD95B58EB5891731
:1008E00018F08EB58F5F85BD82E08ABD81E084BD42
:1008F00080E489BF80E285BB8ABF8BB780628BBFF3
:1009000010923E011092BB0010923C0110923D01EA
:10091000089584B5882379F49091BB00983058F4F9
:100920008DB3E92FF0E0ED54FF4F80839F5F9093EC
:10093000BB0081E084BD80917C0084FF12C0609187
:10094000BB00662321F480913F01882351F083EBA3
:1009500090E0FFDB8091BB00887080933F01109294
:10096000BB0083B7882369F5E0913E0180913D018A
:100970008E1739F1F0E0E454FF4F80816FDF209152
:100980003E012F5F2F7720933E0112BE9BE49EB95C
:100990001EBA982F9295907F9F6098BD8695F89487
:1009A0008FB983E083BF789480918D0087FF09C061
:1009B00080913D018095820F8F77823010F01092E8
:1009C0008D000895FC018381813049F484E590E035
:1009D00090938C0080938B0080915400089586E65C
:1009E00090E090938C0080938B0083E40895FC0149
:1009F0002081822F80768032B9F49181892F8052B4
:100A0000823010F48FEF0895923239F480916E00A5
:100A1000882319F482E080936E0027FD05C081E0F1
:100A200080933F0180E0089580E00895FC0180916B
:100A30006F00808380917000818312821382148200
:100A4000158288E0868387E00895DC010BC0E92FDA
:100A5000F0E0E454FF4F8D9180839F5F9F779093E8
:100A60003D01615090913D01662389F780913E01DF
:100A70008150891B8F77823018F48FEF80938D001F
:100A800008952EE088E190E00FB6F894A89581BD16
:100A90000FBE21BD2EDE8AEF88BB85E087BBA895FF
:100AA00084EC99E02CE931E0F9013197F1F70197F5
:100AB000D9F717BA80EC92E19093700080936F00A1
:100AC000DFDE0FDB10926E0010923F017894A89544
:100AD00044DB1FDF90916E009923C9F38091A7003A
:100AE00084FFF5CF923021F482E690E068E003C005
:100AF0008AE690E062E029DB80916E00815080936D
:100B00006E00E5CFFC01808180936F00818180932E
:100B1000700080916F0090917000B2DE81E00895C6
:100B2000A1E21A2EAA1BBB1BFD010DC0AA1FBB1FF1
:100B3000EE1FFF1FA217B307E407F50720F0A21B63
:100B4000B30BE40BF50B661F771F881F991F1A94D0
:100B500069F760957095809590959B01AC01BD01FA
:100B6000CF010895E199FECF1FBA8EBBE09A992775
:100B70008DB30895262FE199FECF1CBA1FBA8EBB04
:100B80002DBB0FB6F894E29AE19A0FBE0196089534
:040B9000F894FFCF07
:0C0B94005AFFA120000000000200030036
:00000001FF
